:2000000012C02AC029C028C027C026C025C024C023C022C021C020C01FC01EC01DC01CC0C1
:200020001BC01AC01AC011241FBECFEDCDBF10E0A0E6B0E0EAEEF7E002C005900D92A03755
:20004000B107D9F710E0A0E7B0E001C01D92A438B107E1F705D1C7C3D3CF1F920F920FB61C
:200060000F9211248F939F93809160008F5F809360008091600090E087709070009729F4F8
:20008000809170008F5F809370008091600090E08F739070009729F4809160008F5F809365
:2000A0006000809171008F5F809371009F918F910F900FBE0F901F901895EF92FF920F9381
:2000C0001F93CF93DF93182F062F0F7367FF14C090E0880F991F845B9F4FF82E10E0E19946
:2000E000FECFFEBAE09A8DB3602FE7DF1F5FF394123009F4AEC0F3CF66FF08C06AE053D35B
:20010000602FDBDF812F6AE04ED3192F802F90E09C01207330702115310509F447C004FDD3
:2001200023C02EC060916000E199FECF602770E06F737070605070406EBBE09A8DB3890FE2
:2001400069E031D3BA01092E02C0660F771F0A94E2F7FB01E223F323309719F4262B372B7E
:2001600009C0892F8F5FECCF9091730020E030E041E050E01150B0F6995F909373000DC0FE
:20018000112319F420E030E008C0E12FF0E0E859FF4F208130E020FD31600F7C29F063E091
:2001A000220F331F6A95E1F741E004C0110F20E030E040E090E080E063E061504423B1F4E0
:2001C000662391F0E199FECF512F5F5FE12FF0E0E050F040EEBBE09A8DB3782F707C96952F
:2001E0009695972B152F02C0892F8695A02FB0E0FD01EC58FF4FE081442319F4C4E0D0E021
:2002000002C0C5E0D0E0F0E00C2E02C0EE0FFF1F0A94E2F7AC58BF4FEC93442351F0522FAF
:2002200057705E2B5C9353E0369527955A95E1F707C0582F56955695569557705E2B5C93B0
:200240000F5F880F880F880F00FDD0CF662309F0B4CFDF91CF911F910F91FF90EF900895FF
:200260002F923F924F925F926F927F928F929F92AF92BF92CF92DF92EF92FF920F931F93EC
:20028000DF93CF93CDB7DEB72B970FB6F894DEBF0FBECDBF1E010894211C311C82E590E04C
:2002A00088879E012C5F3F4FF101E199FECF8EBBE09A9DB390838F5FE217F30711F031966F
:2002C000F4CF83E481BD7894209172002D83DD24772455245394CC2400E0BB2444244394ED
:2002E000BEE1AB2E18E27E010894E11CF11CA1E08A2E912CA1014C5F5F4F5A874987672C32
:200300007A2C1FC07394809170008150809370005BE35715A0F489819A8101969A83898359
:200320002B813C812115310541F04A9431F4809170008F5F80937000422E1860772401112D
:200340001860809170008823E9F613FFAFC0DD2009F0ACC0662009F0A9C0177DD7018D91C5
:200360009C911197B2E0803D9B0728F0805D9240F70191838083D701ED91FC911197CF0186
:200380006CE370E01CD27F836E832E81CF016CE370E015D2A82E222309F42CE00230D9F1B8
:2003A000033030F4002369F0013009F07FC02FC0043009F45AC00430A0F1053009F076C09E
:2003C0006EC0CC2029F0E1E0CE122A2D822F20C02A3008F42259822F62E46FDEE4E7F0E0B1
:2003E0008081880F880F819320E0EC37F207C1F78091770081608093770080917900816088
:20040000809379008A2D6AE458DE10624FC0872D62E453DE4BC0822F60E54FDE8A2D64E53B
:20042000F8CF8A2D65E0BFD1A82E30E6273018F4622F6F5F02C06DE0621B8D81B4D1273045
:2004400018F0822F8650980F892F6AE0A3D1891B820F632F3B8731DE4D814F5F4D832A2DB5
:200460003B85303619F534E6E1CF822F6AE09BD180937400822F97D1909375008A2D93D1C4
:20048000809377008A2D8FD190937800872D8BD180937A00872D87D190937B0007C085B7D6
:2004A000806585BF89B78D7F89BF1860812F90E0212F207C09F48AC0E4E7F0E0119250E046
:2004C000EC37F507D9F79C012074307086FD03C0CC2009F461C0BB2029F40F5F063008F078
:2004E00062C062C021153105B1F163E0B61631F45394651508F058C0552456C0CC20D9F0C1
:20050000D7012D913C91B1E0CB1619F4245C3F4F0EC0C9010196D70111969C938E936CE39E
:2005200070E04DD1009709F03FC02B533040F7013183208339C0EB2CFF240894E108F108D0
:20054000EE0CFF1C21E030E02C0F3D1FE20EF31ECC24C39428C0CC2039F132E0C316D1F4E8
:200560008885F1019191E199FECF1CBA8EBB9DBB0FB6F894E29AE19A0FBE8F5F49855A85EC
:20058000E417F50779F7CC24BB247E010894E11CF11C0AC0C39408C0B39453E05B1518F421
:2005A00000E0BB2401C000E01F71BB2039F0CC2029F48B2D815062E880DD08C01860BB20F3
:2005C00029F4002319F464E0609371008D2D90E08F709070009761F411BA81B387BB87B396
:2005E0008ABB12BA82B388BB88B38BBBDD2011F0DA94A7CE70E171BB84E082BB80E090E022
:200600008034910511F4106416C09C012F5F3F4FA0E681309A0770F01F7B1068C9018F7075
:200620009070009719F017BA16BA04C0B1E0B8BBE1E1E7BBC901829902C00196E1CF862DAC
:2006400090E0FC01EF59FF4F208122952F70309171003F713093710015FF39C0309171004B
:20066000369536953695313061F0313020F0323071F080E004C08C589F4FDC018C9130E033
:200680000BC0FC01EC58FF4F3081808505C08C589F4FFC01308580E090917100977001C047
:2006A000330F9A95EAF74091710090E0477068E070E0641B7109062E02C0959587950A9414
:2006C000E2F7382B50E840E090E080E006C08C589F4FDC013C91F6CF4F5F652F6323D9F01E
:2006E000E42FF0E0EF59FF4FE081F0E0BF0167707070E3FF08C0F40102C0EE0FFF1F6A955E
:20070000E2F78E2B07C0D40102C0AA0FBB1F6A95E2F79A2BD39456954730F1F6DD2039F0E3
:200720003D2D330FD52CD294E0EFDE22D32ACC2031F03091600031FD02C090E080E0382F85
:200740003095492F409523FF09C02770B82D01C0BB0F2A95EAF73B2B8B2B08C0F40102C05A
:20076000EE0FFF1F2A95E2F74E2B9E2B282F22952695269523702ABB97BB81BB832F829531
:200780008695869583708BBB48BB32BB6394F7E06F22D7CD002480FD060E660F11F08695B1
:2007A000D1F7802D0895991B79E004C0991F961708F0961B881F7A95C9F780950895AA1B5B
:2007C000BB1B51E107C0AA1FBB1FA617B70710F0A61BB70B881F991F5A95A9F78095909581
:1A07E000BC01CD010895F894FFCF01045FDE318BC296A710285445556D00ED
:00000001FF
